:1000000008308A00002800008A1D0A128A190A1680
:100010008A11831A0F28A500030EA6001428831244
:10002000A500030EA600A614A50E0408A70020082C
:10003000A8002108A9002208AA002308AB00240870
:10004000AC0083128C308400001D28280C19F9287C
:10005000270884002808A0002908A1002A08A20077
:100060002B08A3002C08A400260E83008312250E63
:10007000A61883160A1A8A1509000A108A100A118E
:10008000820728340C34013406340A108A100A110D
:10009000820770346934633454344134433448340F
:1000A0004F3400340A108A100A118207563465341E
:1000B00072342E34203431342E34313400340A106A
:1000C0008A100A1182070A340D347034693463349B
:1000D00054344134433448344F34203431342E3492
:1000E0003134203400340A108A100A118207303467
:1000F00033342D344A3441344E342D34393437348A
:1001000000340A108A100A1182070A340D3462344E
:100110007934203443346F347234643420344A34B4
:100120006F34683461346E346E346D3465347934D0
:100130006534723400340A108A100A1182070A34B6
:100140000D340A340D3400340A108A100A11820763
:100150002034723470346D340A340D3400340A1093
:100160008A100A118207203448347A3400340A1085
:100170008A100A11820720342F346D3400340A109B
:100180008A100A1182072534753420343034203423
:10019000723470346D340A340D3400340A108A100D
:1001A0000A1182072D342D342D342D342D342D3465
:1001B0002D342D3400340A108A100A11820720349D
:1001C00020344634723465347134203420340034A1
:1001D0000A108A100A1182072D34203400340A10C4
:1001E0008A100A118207203442346C3420342D34B2
:1001F00000341608AE001508AD008F018E012F14D3
:100200000C118A1128285408031915290130A1005E
:10021000BF30A0006400A00B0A29A10B08294A30B6
:10022000A000A00B1129D40B062900340130660070
:100230008610061186110F30D40003210130D3003F
:1002400004305302031837290330E30063080F39E1
:10025000A000A00E0F3006052004860086150000C1
:1002600086112130A000A00B3329D30A20290230A7
:10027000E30063080F39A000A00E0F30060520042C
:1002800086008615000086112130A000A00B4629AB
:10029000D301043053020318A32953083D20D4008E
:1002A000E0015408E1008610F1306600061586155D
:1002B00000000608A000200E0F39E30086110000A0
:1002C000861500000608A000200E0F39E2008611F6
:1002D000013066006308A000A00EF030A0052008E1
:1002E0006204A100210880390038031D5429E00868
:1002F000031D7C2986107D2986140611861161084C
:10030000E200E20E0F30E2056208E30063080F39F5
:10031000A000A00E0F300605200486008615000000
:10032000861161080F39E2006208E30063080F39A3
:10033000A000A00E0F3006052004860086150000E0
:100340008611D30A49298A15182801305D0203193C
:10035000AC294030DE00AD29DE0101305C02DE0751
:100360005E088038DF00E0015F08E1008610F130B0
:1003700066000615861500000608A000200E0F393D
:10038000E30086110000861500000608A000200E7C
:100390000F39E2008611013066006308A000A00E4C
:1003A000F030A00520086204A1002108803900383F
:1003B000031DB729E008031DDF298610E0298614F4
:1003C000061186116108E200E20E0F30E2056208B4
:1003D000E30063080F39A000A00E0F3006052004CB
:1003E000860086150000861161080F39E200620858
:1003F000E30063080F39A000A00E0F3006052004AB
:10040000860086150000861100345B08A0000C30C1
:1004100020020319142A0A3020020319662A083020
:10042000200203196C2ABE2AE0010130E100861087
:10043000F13066000615861500000608A000200EA3
:100440000F39E30086110000861500000608A000A1
:10045000200E0F39E2008611013066006308A0000B
:10046000A00EF030A00520086204A1002108803908
:100470000038031D182AE008031D402A8610412A6F
:100480008614061186116108E200E20E0F30E205C3
:100490006208E30063080F39A000A00E0F300605C4
:1004A0002004860086150000861161080F39E200DD
:1004B0006208E30063080F39A000A00E0F300605A4
:1004C00020048600861500008611112B0130DC0007
:1004D0000230DD00A521112BE0011030E100861073
:1004E000F13066000615861500000608A000200EF3
:1004F0000F39E30086110000861500000608A000F1
:10050000200E0F39E2008611013066006308A0005A
:10051000A00EF030A00520086204A1002108803957
:100520000038031D702AE008031D982A8610992AB6
:100530008614061186116108E200E20E0F30E20512
:100540006208E30063080F39A000A00E0F30060513
:100550002004860086150000861161080F39E2002C
:100560006208E30063080F39A000A00E0F300605F3
:1005700020048600861500008611112B0130E00052
:100580005B08E1008610F130660006158615000054
:100590000608A000200E0F39E30086110000861522
:1005A00000000608A000200E0F39E200861101307D
:1005B00066006308A000A00EF030A00520086204C9
:1005C000A100210880390038031DC32AE008031D5B
:1005D000EB2A8610EC2A8614061186116108E200C7
:1005E000E20E0F30E2056208E30063080F39A00055
:1005F000A00E0F3006052004860086150000861127
:1006000061080F39E2006208E30063080F39A000B7
:10061000A00E0F3006052004860086150000861106
:10062000112B00341030A000A301DE01DB0CDA0C2A
:10063000031C202B5C08A3070318DE0A5D08DE07F5
:10064000DE0CA30CA20CA10CA00B162B0034560838
:10065000A101550203182F2B5508A0003B2BA00128
:100660000830D700D50DA00D560820020318A000B1
:10067000A10DD70B322B00345418572BD4186B2BE9
:100680005308D5006430D60027232008D300210862
:100690003030031D502B5419572BD4192030522BB6
:1006A0005411D411A10721080C1E542B9900530892
:1006B000D5000A30D60027232008D3002108303087
:1006C000031D662B54196B2BD4192030A107210868
:1006D0000C1E682B99003030D30753080C1E6E2B6C
:1006E00099000034D41B852B0F30A000530EA005B9
:1006F0000A30200203187F2B3030A007812B5408CA
:10070000A00720080C1E822B99000F30D3050A3059
:10071000530203188D2B30308F2BD4135408D3077A
:1007200053080C1E912B99000034A101A201A001D5
:10073000A3015D08031D9F2B5C080319B92B103022
:10074000DE000310DA0DDB0DA00DA30D5D08230202
:10075000031DAC2B5C082002031CB52B5C08A00217
:10076000031CA3035D08A3020314A10DA20DDE0B5D
:10077000A12B0000003457102730D9001030D800CA
:10078000D501053055020318FF2B5408DB00530830
:10079000DA005908DD005808DC0095232108D6004E
:1007A000DB015608DA005908DD005808DC00122386
:1007B0002208A3002108D3022308031CD403D40277
:1007C0005908DB005808DA00DD010A30DC00952307
:1007D0002208D9002108D800D608031D5714571C39
:1007E000F92B30305607DA005A080C1EF52B990009
:1007F000FD2B20300C1EFA2B9900D50AC12B8A152F
:10080000E52D57102730D9001030D800D50105301C
:1008100055020318432C5408DB005308DA0059082A
:10082000DD005808DC0095232108D600DB015608BE
:10083000DA005908DD005808DC0012232208A30062
:100840002108D3022308031CD403D4025908DB0077
:100850005808DA00DD010A30DC0095232208D900AF
:100860002108D800D608031D5714571C3E2C3030E1
:100870005607DA005A08DB000522412C2030DB0045
:100880000522D50A072C8A15002EFF3FFF3FFF3FA8
:10089000FF3FFF3FFF3FFF3FFF3FFF3FFF3FFF3F68
:1008A000FF3FFF3FFF3FFF3FFF3FFF3FFF3FFF3F58
:1008B000FF3FFF3FFF3FFF3FFF3FFF3FFF3FFF3F48
:1008C000FF3FFF3FFF3FFF3FFF3FFF3FFF3FFF3F38
:1010000084019F308400073080000C3083169900E3
:1010100022309800831290309800FF30B000B90160
:10102000BA01BB01BC01C4010030D2008A111629EB
:101030008A150130DC000130DD008A11A5218A15F6
:10104000D30153088A1145208A15003803192E2828
:10105000D30ADB008A1105228A1521280130DC0021
:101060000230DD008A11A5218A15D30153088A11A7
:1010700052208A15003803194328D30ADB008A114D
:1010800005228A153628D30153088A115F208A1554
:10109000D30A0C1E492899000F305302031D44281F
:1010A000D30153088A1173208A15D30A0C1E5628BF
:1010B000990009305302031D5128D30153088A11A6
:1010C00081208A15D30A0C1E63289900153053021B
:1010D000031D5E28D30153088A119B208A15D30A69
:1010E0000C1E7028990004305302031D6B280C302D
:1010F000D300FA30D4008A1103218A15D30B792842
:1011000035309000073097008C3084000015C030D7
:101110008B04AE010030AD002F105010B016300817
:101120006700871A952852109628521430163008F6
:101130006700071A9D28D2109E28D214B0153008D7
:1011400067008719A5285211A628521583168516FF
:101150008312851AAD28D211AE28D21552080F3A43
:10116000D1003F308B058B1BB1282E08CC002D08F9
:10117000CB00C0308B044C084E02031CC7284C081F
:101180004E02031DD7284B084D020318D7284D08DF
:101190004B02A1004C08A0004E08031CA003200233
:1011A000A30021082308840A80008403E6284B0852
:1011B0004D02A1004E08A0004C08031CA003200211
:1011C000A30021082308840A80008403D500A30813
:1011D000031DF528283055020318F52803304F0267
:1011E0000318F4284F08CF0AF7285014CF014C08F1
:1011F000CE004B08CD002F18FF2800300029013009
:10120000D30003304F0203190729003008290130A9
:10121000530500380319272EBD01BE014C08A30158
:10122000BF004B08C000501C4B2950103D08B900AE
:101230003E08BA003F08BB004008BC00C101643052
:10124000C2003B08D6003C08D5004108D400420843
:10125000D30031295308D5070318D60A5408D607F6
:1012600000341030DB005608DA005508D900D601EA
:10127000D501DA0CD90C03182A21D60CD50CD80CC0
:10128000D70CDB0B39295608B9005508BA005808A5
:10129000BB005708BC00C1016430C2003F08D60043
:1012A0004008D5004108D4004208D3005E29530805
:1012B000D5070318D60A5408D60700341030DB00CF
:1012C0005608DA005508D900D601D501DA0CD90C38
:1012D00003185721D60CD50CD80CD70CDB0B66297C
:1012E0005608BD005508BE005808BF005708C0008A
:1012F0003908B1003A08B2003B08B3003C08B4001A
:101300000130C300093043020318C1293908D30052
:101310003A08D4003B08D5003C08D6003108D70075
:101320003208D8003308D9003408DA005A08D60742
:10133000031C9C290130D507031CA0290130D407C8
:10134000031CA4290130D3075908D507031CAA2977
:101350000130D407031CAE290130D3075808D40745
:10136000031CB4290130D3075708D3075308B90029
:101370005408BA005508BB005608BC004308C30A0D
:1013800082293908D3003A08D4003B08D5003C082C
:10139000D6003D08D7003E08D8003F08D9004008D5
:1013A000DA005A08D607031CD7290130D507031CD9
:1013B000DB290130D407031CDF290130D30759088A
:1013C000D507031CE5290130D407031CE9290130A6
:1013D000D3075808D407031CEF290130D307570857
:1013E000D3075308B9005408BA005508BB00560883
:1013F000BC00C1010A30C2003908D3003A08D40049
:101400003B08D5003C08D6004108D7004208D80068
:10141000DA01DB01D901530DDB0D5808DB02570857
:10142000031C570FDA020001031C0130D902D30D4F
:101430000730DC00530DDB0DDA0DD90D5808531CB5
:101440002B2ADB025708031C570FDA020001031C8A
:101450000130D902342ADB0757080318570FDA077F
:10146000000103180130D907D30DDC0B1A2A540DE3
:10147000DB0DDA0DD90D5808531C482ADB0257083A
:10148000031C570FDA020001031C0130D902512A54
:10149000DB0757080318570FDA070001031801305C
:1014A000D907D40D0730DC00540DDB0DDA0DD90D52
:1014B0005808541C652ADB025708031C570FDA0230
:1014C0000001031C0130D9026E2ADB0757080318FC
:1014D000570FDA07000103180130D907D40DDC0BD0
:1014E000542A550DDB0DDA0DD90D5808541C822AEB
:1014F000DB025708031C570FDA020001031C0130FE
:10150000D9028B2ADB0757080318570FDA070001A7
:1015100003180130D907D50D0730DC00550DDB0D60
:10152000DA0DD90D5808551C9F2ADB025708031CF9
:10153000570FDA020001031C0130D902A82ADB0789
:1015400057080318570FDA07000103180130D907AD
:10155000D50DDC0B8E2A560DDB0DDA0DD90D580892
:10156000551CBC2ADB025708031C570FDA02000186
:10157000031C0130D902C52ADB0757080318570F8F
:10158000DA07000103180130D907D60D0730DC0057
:10159000560DDB0DDA0DD90D5808561CD92ADB0281
:1015A0005708031C570FDA020001031C0130D9024F
:1015B000E22ADB0757080318570FDA070001031860
:1015C0000130D907D60DDC0BC82A5618ED2A580869
:1015D000DB0757080318570FDA075308B9005408F8
:1015E000BA005508BB005608BC003908B5003A08D7
:1015F000B6003B08B7003C08B800C1013230C20059
:101600003508D3003608D4003708D5003808D6008E
:101610004108D7004208D8005808D607031C122BEF
:101620000130D507031C162B0130D407031C1A2BDD
:101630000130D3075708D507031C202B0130D407EE
:10164000031C242B0130D3075308B5005408B600FF
:101650005508B7005608B800C1016430C20035080B
:10166000D3003608D4003708D5003808D600410822
:10167000D7004208D800DA01DB01D901530DDB0D98
:101680005808DB025708031C570FDA020001031C3D
:101690000130D902D30D0730DC00530DDB0DDA0D1C
:1016A000D90D5808531C5E2BDB025708031C570F3B
:1016B000DA020001031C0130D902672BDB0757084F
:1016C0000318570FDA07000103180130D907D30DAB
:1016D000DC0B4D2B540DDB0DDA0DD90D5808531CC6
:1016E0007B2BDB025708031C570FDA020001031C97
:1016F0000130D902842BDB0757080318570FDA078C
:10170000000103180130D907D40D0730DC00540D57
:10171000DB0DDA0DD90D5808541C982BDB02570845
:10172000031C570FDA020001031C0130D902A12B60
:10173000DB0757080318570FDA07000103180130B9
:10174000D907D40DDC0B872B550DDB0DDA0DD90D28
:101750005808541CB52BDB025708031C570FDA023C
:101760000001031C0130D902BE2BDB075708031808
:10177000570FDA07000103180130D907D50D0730DC
:10178000DC00550DDB0DDA0DD90D5808551CD22B98
:10179000DB025708031C570FDA020001031C01305B
:1017A000D902DB2BDB0757080318570FDA070001B4
:1017B00003180130D907D50DDC0BC12B560DDB0DFD
:1017C000DA0DD90D5808551CEF2BDB025708031C06
:1017D000570FDA020001031C0130D902F82BDB0796
:1017E00057080318570FDA07000103180130D9070B
:1017F000D60D0730DC00560DDB0DDA0DD90D58087B
:10180000561C0C2CDB025708031C570FDA02000190
:10181000031C0130D902152CDB0757080318570F9A
:10182000DA07000103180130D907D60DDC0BFB2BBA
:101830005618202C5808DB0757080318570FDA07EB
:101840005308B5005408B6005508B7005608B8004C
:101850005108A00020080319522C0130200203195E
:101860005A2C023020020319622C03302002031983
:101870006A2C043020020319722C0530200203194F
:101880007B2C063020020319832C07302002031919
:101890008B2C083020020319942C093020020319E4
:1018A0009C2CA42CB1011E30B2008430B3008030D7
:1018B000B400AC2C0730B1002730B2000E30B300BA
:1018C000B401AC2C0330B1009330B2008730B300C8
:1018D000B401AC2C0230B1006230B2005A30B30017
:1018E000B401AC2C0130B100C930B200C330B30038
:1018F0008030B400AC2C0130B1006E30B200363014
:10190000B300B401AC2C0130B1003130B2002D3045
:10191000B300B401AC2C0130B1000530B2009430FA
:10192000B3004930B400AC2CB101E430B200E13076
:10193000B300C030B400AC2CB101CB30B200733076
:10194000B3005530B400AC2C0330B1009330B2007A
:101950008730B300B401AC2C3108D3003208D40076
:101960003308D5003408D6003708D7003808D80027
:10197000DA01DB01D901530DDB0D5808DB025708F2
:10198000031C570FDA020001031C0130D902D30DEA
:101990000730DC00530DDB0DDA0DD90D5808531C50
:1019A000DB2CDB025708031C570FDA020001031C73
:1019B0000130D902E42CDB0757080318570FDA0768
:1019C000000103180130D907D30DDC0BCA2C540DCC
:1019D000DB0DDA0DD90D5808531CF82CDB02570823
:1019E000031C570FDA020001031C0130D902012D3C
:1019F000DB0757080318570FDA07000103180130F7
:101A0000D907D40D0730DC00540DDB0DDA0DD90DEC
:101A10005808541C152DDB025708031C570FDA0217
:101A20000001031C0130D9021E2DDB0757080318E3
:101A3000570FDA07000103180130D907D40DDC0B6A
:101A4000042D550DDB0DDA0DD90D5808541C322D1F
:101A5000DB025708031C570FDA020001031C013098
:101A6000D9023B2DDB0757080318570FDA0700018F
:101A700003180130D907D50D0730DC00550DDB0DFB
:101A8000DA0DD90D5808551C4F2DDB025708031CE1
:101A9000570FDA020001031C0130D902582DDB0771
:101AA00057080318570FDA07000103180130D90748
:101AB000D50DDC0B3E2D560DDB0DDA0DD90D58087A
:101AC000551C6C2DDB025708031C570FDA0200016E
:101AD000031C0130D902752DDB0757080318570F77
:101AE000DA07000103180130D907D60D0730DC00F2
:101AF000560DDB0DDA0DD90D5808561C892DDB0269
:101B00005708031C570FDA020001031C0130D902E9
:101B1000922DDB0757080318570FDA070001031847
:101B20000130D907D60DDC0B782D56189D2D58089D
:101B3000DB0757080318570FDA075308B10054089A
:101B4000B2005508B3005608B400A3013308D5000D
:101B50002308D6005608DB005508DA000130DD0006
:101B60000030DC008A1112238A152208D4002108D3
:101B7000D300A30134085307C50023080318013E0E
:101B80005407C6005108D3000C30D4008A113C23FE
:101B90008A1520300C1ECA2D99004C08D30037300E
:101BA000D4008A1172238A154B08D3003730D40031
:101BB0008A1172238A1520300C1EDC2D99004608EC
:101BC000D4004508D3008A11BB2B8A15D3015308D2
:101BD0008A11A4208A15D30A0C1EEC2D9900063018
:101BE0005302031DE72D0130DC000230DD008A11B5
:101BF000A5218A154608D4004508D3008A11012C76
:101C00008A155108A00020080319072E162ED301AB
:101C100053088A11AF208A1500380319152ED30AEC
:101C2000DB008A1105228A15082E252ED3015308C0
:101C30008A11B7208A1500380319242ED30ADB0035
:101C40008A1105228A15172E252E2F10652E510870
:101C5000D3000C30D4008A113C238A1520300C1E8E
:101C60002F2E99000430D30030300C1E352E9900F1
:101C7000D30B342E0530D30020300C1E3D2E99009E
:101C8000D30B3C2E0330D30053088A11BF208A1592
:101C9000D30A0C1E492E99000A305302031D442E0C
:101CA0000130DC000230DD008A11A5218A15D30144
:101CB00053088A11CE208A1500380319652ED30ADD
:101CC000DB008A1105228A15582E5108A000200831
:101CD00003196B2E812E0130DC000130DD008A11EA
:101CE000A5218A15D30153088A11DB208A150038F3
:101CF0000319802ED30ADB008A1105228A15732E60
:101D0000AD2E0130DC000130DD008A11A5218A15DD
:101D1000D30153088A11E8208A1500380319962E3A
:101D2000D30ADB008A1105228A15892E303051072B
:101D3000D3005308DB008A1105228A15D30153080A
:101D40008A11EF208A1500380319AC2ED30ADB0064
:101D50008A1105228A159F2EAD2EC830D4008A1113
:101D600003218A158E286300FF3FFF3FFF3FFF3F9F
:101D7000FF3FFF3FFF3FFF3FFF3FFF3FFF3FFF3F73
:101D8000FF3FFF3FFF3FFF3FFF3FFF3FFF3FFF3F63
:101D9000FF3FFF3FFF3FFF3FFF3FFF3FFF3FFF3F53
:101DA000FF3FFF3FFF3FFF3FFF3FFF3FFF3FFF3F43
:02400E00F13F80
:00000001FF
